:1000000009C018951895189518951895189518956C
:10001000189518958FE98DBFC0E8E8E74E2EDD27CB
:100020005D2EEEE3F0E0A0E6B0E088278D933197F7
:10003000E9F76624BA9AB99ABB9880E184BB82E258
:1000400087B980E886B9C39AC198C29A81E0882EA0
:10005000BB98AFEF9C9197FF04C0B39B0EC09F77F6
:100060009C93B3990AC089E19F939927A2D09F914D
:10007000B39903C090689C9303D0EACFF894FFCF64
:10008000A8E00C9141E0041709F00BC059D09B2C5B
:1000900091E0A9E09DD0C29888EC90E08AD0C29A05
:1000A0001DC0A8E00C9142E0041709F017C048D029
:1000B000AB2C91E0AAE08CD0092D4A2D040FC02E64
:1000C000C29888EC90E075D0C29A88EC90E071D02C
:1000D000C29888EC90E06DD0C29A3FC08394A8E0AB
:1000E0000C9142E0041710F009F001C002C081E059
:1000F000882E089580E0A82E80E0982E80E0C82EFB
:1001000081E0882EC29888EC90E053D0C29A88ECA7
:1001100090E04FD0C29888EC90E04BD0C29A88EC27
:1001200090E047D0C29888EC90E043D0C29A88EC27
:1001300090E03FD0C29888EC90E03BD0C29A83CF49
:10014000369A0027A6E28C9186FB0EF401E040E08F
:10015000041709F0F6CFB5B00895F2DFABE00C91CB
:10016000ACE04C91041710F009F001C002C0C19A34
:1001700001C0C198BB98AFEF9C9197FF04C0B39B9F
:100180000EC09F779C93B3990AC089E19F939927EA
:1001900010D09F91B39903C090689C93ABCFDDCFF3
:1001A0003197F1F70895689462F80895E89462F839
:1001B0000895EF93FF93EE27E82BE92B31F0E0E66B
:1001C000F9E03197F1F70197D1F7FF91EF91089599
:1001D000903029F08C9186959A95E9F78C93089543
:00000001FF
